:10000000020E5B022003000000000002200B000033
:10001000000000022013000000000002087200002F
:100020000000000220232165216E21D721F44144E4
:10003000415561A8411BA16FA16B41E541D3A129A5
:10004000020F5C219321B4434F5059524947485401
:1000500020284329203139383120494E54454C203D
:10006000434F52504F524154494F4E20414C4C2027
:100070005249474854532052455345525645449897
:10008000C99B89A2A3A4A58082C8E0A10A0BC2A82B
:10009000A9C0AAABA0D59990919293949596978474
:1000A00081ACB09AC1CAAD0CAE0DE186CB414343E1
:1000B00020414C4C204220202042522020425230ED
:1000C0002042523120425232204252332043425980
:1000D000544442595444495350444F574E44505449
:1000E00052464F524546524F4D474F2020494520DA
:1000F00020495020204D474F2050312020503320A0
:10010000205043202050524F475053572052302008
:1001100020523120205232202052332020523420CD
:10012000205235202052362020523720205242497A
:10013000545242595453434F4E53454E445350200A
:1001400020535445505355425254434F4E54494CFA
:100150004C544D4F44544F202055504C4F58425909
:100160005458464552EA3099FDF599C29922309883
:10017000FDE599C2E7C298641B7006120EB7020F24
:1001800007641BB461004007B47B005002C2E52243
:10019000A29822C083C082902FA3C0A8C2ACE0C0A6
:1001A000E0741BF0D0E0D0A8D082D083B41B0280D2
:1001B000E2C2E722C083C082E0D082D083C2E7647B
:1001C0001BC36001B3223099FD22902F94E0308F41
:1001D000FDC28FD5E0F822C2B431CA31CAEA7A0A28
:1001E000D31392B4C0E031CA31CAD0E0DAF2227A35
:1001F0002031652230B5FD20B5FD31CA20B5F57539
:10020000258031CA31CAA2B5C52513C52550F331A1
:10021000CA31CA30B5DEE525C2E7227A0D31657AEA
:100220000A3165227A0D31D77A0A31D722EA540F82
:100230002490D43440D4FA20D50331652231D7221A
:10024000D2D58002C2D5EAFCC4FA512DECFA512D68
:1002500022D2D58002C2D55146EBFA5146227842CD
:100260007530049000A9EAC0E07A01120EE1D0E0F6
:10027000FA75F004EAA42582F582E5F03583F5836A
:10028000E4938631B53109A308D530F475410122D4
:100290005004754103227541022278427530049062
:1002A00000A9EAC0E07A01120EE1D0E0FA75F0048C
:1002B000EAA42582F582E5F03583F583E6B42002D1
:1002C0008007F531E493B53107A308D530EEE42279
:1002D00074FF228A838B82E493FF6008E4A393FA7D
:1002E0003165DFF822780090007FE8936A600408A7
:1002F000B82EF49000ADE875F004A42582F582E5EF
:10030000F03583F5837800E893FA64206006316560
:1003100008B804F322EBC0E051E57A3D3165D0E046
:10032000FA514431EF22902FA5E0FE902FA4E0FF78
:100330006E705C7E007F00902FA6316EB47F18BF78
:1003400000067A07316580F27A08316531EF7A0864
:1003500031651F158280E3B41804511B80D5B41297
:1003600018511BEF60D48582F07582A6E0FA3165E2
:10037000A3E58265F070F580C1BF50067A0731654C
:1003800080B8F0FA0FE0A3640D6004316580AB9093
:100390002FA6E5822EF582E0F5F00E902FA5EEF067
:1003A000902FA4EFF0E5F022E527B420067126F5A2
:1003B0002780F57529047842FA12053B40030204B0
:1003C0007F120551501CA62708882F7126F527A8F3
:1003D0002FAA27D529EB120551500D7126F527FAC2
:1003E00080F4762008D529FA75320175332DEAC0DC
:1003F000E07A07120EE1D0E0FAE533C39532402CE3
:10040000E5322533C313F534FA515EE541B40207F2
:10041000E53414F53380E2B40307E53404F53280A3
:10042000D8E53404F53224FEF53380CDE53304C33A
:100430009532403DE543B42003020F61753201154A
:1004400034AA34519A700515328534330534AA34F0
:10045000519A7006D532178534330534AA34519A2F
:100460007006D53209853433853334D53203020F13
:100470006190007E7A02120EE1E53493F536221285
:100480000546504875380075390012055E502E1229
:10049000054650257B30E53975F010A4F539E52780
:1004A000C39B2539F539AAF075F010E538A42AF573
:1004B000387126F527AA2780D17B3780D9E527B464
:1004C00048047126F527753601E536228A369004F0
:1004D000EEEAC0E07A03120EE1D0E0FAE493601E87
:1004E000B53607A3E493F536801AA3A380EE2C0259
:1004F0002F033D042B093B0623080D07000075362A
:1005000000020F61BA0D06752720E536227126F527
:1005100027E5362271A8B401162271A8B40110E5AE
:10052000386003020F6CE5362271A8B4070122027D
:100530000F61EA30E6022409540F22EAB45B00504E
:1005400004B44000B322EAB43A005004B43000B31B
:1005500022EAB45B005004B44000B350E922EAB48C
:1005600047005004B44100B350DC22C2D58002D20F
:10057000D5E52E7013852C82852B8320D505E49339
:10058000020618EAF0020618B40121E52B7006E510
:100590002C54F86003020619902F82E05418252C81
:1005A000F58220D503E08070EAF0806CB40219E592
:1005B0002B7066E52C20E76175832F852C8220D572
:1005C00003E08054EAF08050B40438E52B704AE52B
:1005D0002C20E74575F00884242075832FF582E0F0
:1005E00005F020D50AD5F0045401802C0380F613C1
:1005F000D5F0FC8AF0A2F0852CF005F033D5F0FCA4
:10060000F0801564066003020F5C852C82852B83C5
:1006100020D503E08002EAF022020F6CB11AAA3959
:10062000B16F71A8B4021B71A8B40704511B71A863
:10063000B4010F052CE52C70E5052BE52B70DF02CE
:100640000F6CB4070122020F617532013190500224
:10065000316EE53BC3952CE53A952B402ED53218EB
:10066000511B7480252EFA51E531EFAA2BAB2C518A
:10067000557A3D3165753210B16BFA514431EF0551
:100680002CE52C70C7052BE52B70C122B4044EB1AC
:100690001AAA39B16FE52CC3953BE52B953A500A60
:1006A000052CE52C70EB052B80E7B1292285362E31
:1006B000532E07B11485382B85392C85383A853966
:1006C0003B71A8B40404D11C8012B40D0AB1148586
:1006D000383A85393B71A8B407B2D14922020F617B
:1006E000E53664896003020F6171A8B4071F7A3D83
:1006F0003165902F87E0FAA3E0FBC082C08351559B
:1007000031EFD083D082A3E582B48FE922E536644D
:10071000046003020F61902F87E4F0A3E582B48F99
:10072000F8753200B114902F87E5822532F582E505
:1007300038F0A3E539F071A8B40702800FB40209BC
:1007400005320532E532B408DB020F6122EA75F0AA
:1007500003A490075673E5A822E5B822E59022E5A8
:10076000B022E59822E58822E58922EA75F004A402
:1007700090077473EBF5A822EBF5B822EBF5902205
:10078000EBF5B022EBF59822EBF58822EBF5892208
:10079000E5365407C0E071A8B4070D7A3D3165D045
:1007A000E0FAF14DFA514422B40414B114E5386072
:1007B00003020F6CD0E0FAE539FBF16BB12922029C
:1007C0000F6171A8B4070D7A3D3165D083D082E006
:1007D000FA514422B4040CB11AE539D083D082F026
:1007E000B12922020F61902F82E05418FAE53654A5
:1007F000072AC0E0C08380CAE536540390080993F5
:10080000C0E075832FC08380B981828380E5365430
:1008100007F537902F8325E02582C0E0C0831203BF
:10082000A8B407237A3D120165E537700DD0E0D0FA
:10083000E0120941FBE5F0FA8009D083D082E0FAAA
:10084000A3E0FB12025522E536B40423120514E599
:1008500037700DD0E0D0E0AA38AB39120950800BC8
:10086000D083D082E538F0A3E539F01205292202C1
:100870000F5CC2AFC082C083902F8FF0902F91E0A9
:1008800064037007D083D082020A98902F8FE09083
:100890002F81F0758282E5D0F0758280E5F0F075E9
:1008A0008284E5A8F0758285D0E0F00582D0E0F082
:1008B000758283E581F075820075D000E8F07801DB
:1008C000A3E6F008B880F9902F91E0F5F075A80044
:1008D000758107120EB7E5F0B40203020CEF700346
:1008E000020C8EB40103020F00020AA0C2AF902FC7
:1008F00091E0D2AB7002C2AB120941902F97F0E5A4
:10090000F01582F0787F902F7FE0F61582D8FAE01C
:10091000F6758284E0E5A8758280E0F5F075828244
:10092000E0F5D0758283E0F581758285E0C0E00551
:1009300082E0C0E0758281E0D082D083C2BBD2AFBA
:1009400032902F83E014F582E0F5F0A3E0C5F022A9
:10095000902F83E014F582EBF0A3EAF0227A0412E0
:100960000EE112021B7AA01202E57A3D12016531F6
:1009700041AAF0FB1202551201EF7A9B902F80E002
:10098000FB1203157A98902F81E0FB1203157A99D8
:10099000902F82E0FB1203157AA11202E57A3D1234
:1009A0000165902F85E0FAA3E0FB1202557A0A7BDD
:1009B000091202D3E590FA1202447A0A7B0E12025F
:1009C000D3E5B0FA1202441201EF1201EF7A52128B
:1009D00001657A42120165902F82E00303035403FC
:1009E000FA12022D7A3D120165902F82E05418F51B
:1009F00082E0FAC082C0831202441201EFD083D099
:100A000082A3E582540770E922042050313D04207E
:100A100050333DE536B4C014120514120529742B69
